:10000000FF0C050040000600070026000B0C220034
:10001000F00C2600F30A050CE201F10C2600F30AAD
:10002000170A0000040CA200F20C2600F30A100CC0
:100030002400FF0C2000A40284061A0A100C2900D8
:10004000200C2A00090C24000402890F4307F30A3C
:100050000002100F4307F30A150C20000902150FC8
:100060004307F30AA4020002200F4307F30A000C1F
:100070002400A50C0002000F4307F30A000C240023
:100080001F0C3F00200C24003F0C3F00400C2400BC
:100090005F0C3F00600C24007F0C3F00000C24002C
:1000A0001F021F0F4307F30A200C24001F023F0FFB
:1000B0004307F30A400C24001F025F0F4307F30AB3
:1000C000600C24001F027F0F4307F30A000C24007A
:1000D000450C2F00600C2400540C2F00400C240011
:1000E0000F02540F4306770AF30C2600F30A000CA4
:1000F0002400040C2900E900E900E900E900E90016
:100100000902FF0F4307F30AA902A9020902010F1E
:100110004307F30A6900A50C2901A903F00C690142
:1001200069025A0CA9010902F50F43069A0AF40C58
:100130002600F30A230C2900E10CE9010307F30A66
:10014000020CA9000307F30A340CA9000306F30A02
:100150000902CE0F4307F30A340C29000F0CE90102
:100160000306F30A2307F30A010CA9000307F30AA5
:100170002307F30AFF0CA9000306F30A2306F30A78
:100180000902430F4307F30AE00C26000502290089
:10019000230C2A006B006C00090203040A06EB0121
:1001A0002B032C032A06EB012B032C034A06EB013D
:1001B0002B032C036A06EB012B032C038A06EB01AD
:1001C0002B032C03AA06EB012B032C03CA06EB011D
:1001D0002B032C03EA06EB012B032C030C02260055
:0801E0000B022700C60AF30A16
:00000001FF
